:1009B800120100020000004005161080010001022B
:1009C80000010A06000200000040010009022000A0
:1009D800010100A0320904000002FF000000070521
:1009E8000202000200070586020002000902200038
:1009F800010100A0320904000002FF000000070501
:100A080001024000000705810240000004030904B8
:100A180026034100430043004500530020004900DD
:100A28002F004F002000500072006F006400750016
:100A380063007400730026035500530042002D0024
:100A48004900440049004F002D00310036002000C5
:0E0A5800460061006D0069006C00790000002E
:03004300020900AF
:030053000209009F
:10090000020F3700020FBC00020FA600020F8E007C
:100910000208C600020D87000200420002005200D9
:100920000208FF000210630002106400021065005C
:1009300002106600021067000210680002106900D1
:1009400002106A000200520002106B0002106C00DC
:1009500002106D0002106E0002106F000210700095
:100960000210710002005200020052000200520008
:100970000210720002107300021074000210750061
:100980000210760002107700021078000210790041
:1009900002107A0002107B0002107C0002107D0021
:1009A00002107E0002107F00021080000210810001
:0809B000021082000210830016
:0A00360000010202030304040505A3
:03000B00020F16CB
:100F1600C0E00509E50970020508640F4508700E72
:100F2600050DE50D7002050C750800750900D0E089
:010F36003288
:100A6600E4F524F523F522F521C203C200C202C231
:100A7600011207F2750E09750FB87516097517CAB2
:100A8600750A09750BD47514097515F475180A7568
:100A96001914D2E843D82090E668E04409F090E6BD
:100AA6005CE0443DF0D2AFD204120E8F90E680E0B7
:100AB60054F7F0538EF8C2033001051203E3C20166
:100AC6003003291200405024C20312000E200016E3
:100AD60090E682E030E704E020E1EF90E682E03045
:100AE600E604E020E0E4120EBE1208FD120BFD80C3
:010AF600C738
:1003E30090E6B9E07003020494147003020511242B
:1003F300FE700302059424FB700302048E14700341
:10040300020488146073146076240560030205F304
:1004130012105B40030205FF90E6BBE024FE60225E
:1004230014603324FD601114602224067048E50E25
:1004330090E6B3F0E50F8037E51690E6B3F0E517E5
:10044300802DE51090E6B3F0E5118023E51290E6E8
:10045300B3F0E513801990E6BAE0FF120EEAAA069C
:10046300A9077B01EA494B600DEE90E6B3F0EF90EC
:10047300E6B4F00205FF0205F812100E0205FF12A2
:10048300103F0205FF1200030205FF120FFC0205D5
:10049300FF12105D40030205FF90E6B8E0247F6081
:1004A3001514601924027063A200E43325E0FFA24F
:1004B30002E4334F8041E490E740F0803F90E6BC94
:1004C300E0547EFF7E00E0D394807C0040047D01F5
:1004D30080027D00EC4EFEED4F2436F58274003E23
:1004E300F583E493FF3395E0FEEF24A1FFEE34E6BA
:1004F3008F82F583E0540190E740F0E4A3F090E6A7
:100503008AF090E68B7402F00205FF0205F81210E0
:100513005F40030205FF90E6B8E024FE6016240264
:1005230060030205FF90E6BAE0B40105C2000205CC
:10053300FF0205F890E6BAE0705590E6BCE0547E01
:10054300FF7E00E0D394807C0040047D0180027D27
:1005530000EC4EFEED4F2436F58274003EF583E445
:1005630093FF3395E0FEEF24A1FFEE34E68F82F58F
:1005730083E054FEF090E6BCE05480131313541F41
:10058300FFE0540F2F90E683F0E04420F0806D806D
:1005930064121061506690E6B8E024FE60192402EC
:1005A300705A90E6BAE0B40104D200804F90E6BAE4
:1005B300E064026047803E90E6BCE0547EFF7E002C
:1005C300E0D394807C0040047D0180027D00EC4EEA
:1005D300FEED4F2436F58274003EF583E493FF333A
:1005E30095E0FEEF24A1FFEE34E68F82F5838008C9
:1005F300120056500790E6A0E04401F090E6A0E018
:030603004480F040
:0106060022D1
:0300330002004E7A
:04004E0053D8EF3262
:100B83005553422D4949524F2D3136005553422D6D
:100B930049492D3136005553422D524F2D313600E0
:100BA3005553422D4949524F2D38005553422D4933
:100BB300492D38005553422D4949524F2D303400A9
:100BC3005553422D4944494F2D3136005553422D3B
:100BD30049444F2D3136005553422D4944494F2D39
:100BE30038005553422D4944494F2D340055534243
:0A0BF3002D49492D4F54484552008A
:040046000233000081
:04104F0043B1402247
:0410530053B1BF22B4
:0410570063B140221F
:0A10200090E740E0F580A3E0F590B2
:07102A0053B1F543B10A22A6
:0E103100C28C538EF75389F1438901C2A92264
:060C5B008B258A26892783
:100C6100E4F528120FE78F29E52925E02402900AEF
:100C71003EF0E4F528AF29EF3395E0FEC3E5289F68
:100C8100EE6480F87480985027AB25AA26A92785A1
:100C9100288275830012070FFDE52875F002A42450
:100CA10040F9740A35F08982F583EDF0052880C595
:010CB1002220
:1007F20012104790E678E05410C4540F4450F53A72
:1008020013E433F53E7AE779407F40AB077D017F01
:10081200037E00120CB290E740E0541FF53C9009B1
:10082200C2E0453CF0E53C540F1207B30850000803
:1008320058010860020868040870050878060880F4
:100842000808880A08900C08980E000008A07BFF90
:100852007A0B7983804E7BFF7A0B798F80467BFF00
:100862007A0B7999803E7BFF7A0B79A380367BFFE6
:100872007A0B79AE802E7BFF7A0B79B780267BFFCD
:100882007A0B79C3801E7BFF7A0B79CF80167BFFB0
:100892007A0B79DA800E7BFF7A0B79E580067BFF93
:1008A2007A0B79F0120C5B121031D2007580FF7551
:1008B20090FF75B2FF75B3FF75B18A75B67F1210DE
:0408C2005302102AA3
:100FD20085388085399012102AE4F50CF50DF50854
:050FE200F509C28C229C
:100BFD00D3E50D9537E50C95364003120FD2E53B45
:100C0D00603AE4F50CF50DE5344533700675332F78
:100C1D007534FFE534153470021533E53445337002
:100C2D0004F53B800FAE33AF347C0B7DFF12075EB6
:100C3D00EF20E005121053800312104FE5B190E63E
:0D0C4D008020E705E04408F022E054F7F0B5
:010C5A002277
:02004000D322C9
:0208FD00D32204
:02105B00D3229E
:0800030090E6BAE0F53DD322BE
:100FFC0090E740E53DF0E490E68AF090E68B04F053
:02100C00D322ED
:08103F0090E6BAE0F535D3227A
:10100E0090E740E535F0E490E68AF090E68B04F048
:02101E00D322DB
:02105D00D3229C
:02105F00D3229A
:02106100D32298
:10005600753B0190E678E05410FFC4540F4450F508
:100066003A13E433F53E90E6B9E01207B30202070D
:1000760001821001A01101B412021F2002252102E3
:10008600252303E12803E12C03E12D03E12E00B92A
:100096002F01CD3001CD31025DA2025DA30257A929
:1000A600022DAC03E1F000ECF100F9F203E1F300FC
:1000B6000003DF90E6BBE0FE90E6BAE07C00240099
:1000C600F537EC3EF53690E6BDE0F53990E6BCE056
:1000D600F538E53745367007C28CC2A9020225D22B
:1000E6008CD2A902022590E6BAE0F580A3E0F5904D
:1000F60002022590E6BEE0752700F528A3E0FEEE95
:100106004227E5284527700490E68BF0E528452729
:1001160070030203E190E6A0E020E1F9C3E528942C
:1001260040E5279400500885272985282A800675EA
:100136002900752A40E4F52BF52CC3E52C952AE514
:100146002B9529501DAF2CC3E5289FFE74402FF533
:1001560082E434E7F583EEF0052CE52C70DC052B04
:1001660080D8E490E68AF090E68BE52AF0C3E5288D
:10017600952AF528E5279529F527809090E6BEE093
:10018600D3940050030203E1E090E68BF090E6A0E2
:10019600E020E1F91210200203E190E740E580F04B
:1001A600A3E590F0A3E5A0F0A3E5B0F0801690E6F5
:1001B600BEE0D3940050030203E190E6A0E020E104
:1001C600F9121020E4802F90E740E580F0A3E59037
:1001D600F0A3E5A0F0A3E5B0F0E5B130E0047F01BF
:1001E60080027F0090E6BAEFF090E7457469F0E48C
:1001F600A3F0A3F0A3F090E68AF0801D90E6BAE0A3
:10020600FF120EEAAA06A9077B01EA494B6008EE2F
:1002160090E6B3F0EF8033D32290E6BEE08001E4AF
:1002260090E68BF00203E190E6B5E054FEF090E62E
:10023600BFE090E68AF090E6BEE090E68BF090E6AE
:10024600BBE090E6B3F090E6BAE090E6B4F00203C5
:10025600E1753E01433A0190E6BAE0752500F526C0
:10026600A3E0FEEE422590E6BEE0752700F528A342
:10027600E0FEEE422790E6B8E064C0600302034960
:10028600E528452770030203E190E6A0E020E1F9A6
:10029600C3E5289440E5279400500885272985283A
:1002A6002A8006752900752A4090E6B9E0B4A33580
:1002B600E4F52BF52CC3E52C952AE52B9529505E04
:1002C600E526252CF582E525352BF583E0FF7440E0
:1002D600252CF582E434E7F583EFF0052CE52C7048
:1002E600D4052B80D0E4F52BF52CC3E52C952AE517
:1002F6002B952950187440252CF582E434E7F583B4
:1003060074CDF0052CE52C70E1052B80DDAD2A7A45
:10031600E779407F40AB07AF26AE25120CB2E490DA
:10032600E68AF090E68BE52AF02526F526E52935BE
:1003360025F525C3E528952AF528E5279529F527E6
:1003460002028690E6B8E0644060030203E1E52815
:10035600452770030203E1E490E68AF090E68BF00D
:1003660090E6A0E020E1F990E68BE0752900F52AF9
:1003760090E6B9E0B4A335E4F52BF52CC3E52C954E
:100386002AE52B952950367440252CF582E434E76E
:10039600F583E0FFE526252CF582E525352BF5834B
:1003A600EFF0052CE52C70D4052B80D0AD2A7AE72A
:1003B60079407F40AB07AF26AE25120DF4E52A251E
:1003C60026F526E5293525F525C3E528952AF528B8
:0C03D600E5279529F527020354D322C324
:0103E20022F8
:100F3700C0E0C083C08290E6B5E04401F0D201531F
:0F0F470091EF90E65D7401F0D082D083D0E0325C
:100FA600C0E0C083C0825391EF90E65D7404F0D038
:060FB60082D083D0E0327E
:100FBC00C0E0C083C0825391EF90E65D7402F0D024
:060FCC0082D083D0E03268
:1008C600C0E0C083C08290E680E030E70E850A1063
:1008D600850B11851412851513800C85141085154A
:1008E60011850A12850B135391EF90E65D7410F093
:0708F600D082D083D0E03274
:100F8E00C0E0C083C082D2035391EF90E65D740837
:080F9E00F0D082D083D0E032D4
:100D8700C0E0C083C08290E680E030E70E850A109D
:100D9700850B11851412851513800C851410851584
:100DA70011850A12850B135391EF90E65D7420F0BD
:070DB700D082D083D0E032AE
:01004200328B
:01005200327B
:0108FF0032C6
:01106300325A
:011064003259
:011065003258
:011066003257
:011067003256
:011068003255
:011069003254
:01106A003253
:01106B003252
:01106C003251
:01106D003250
:01106E00324F
:01106F00324E
:01107000324D
:01107100324C
:01107200324B
:01107300324A
:011074003249
:011075003248
:011076003247
:011077003246
:011078003245
:011079003244
:01107A003243
:01107B003242
:01107C003241
:01107D003240
:01107E00323F
:01107F00323E
:01108000323D
:01108100323C
:01108200323B
:01108300323A
:060CFA00AB07AA06AC05E1
:100D0000E4FDE53E600F7E000DEE2400F582E43444
:100D100000F583EAF0AE050D74002EF582E4340090
:100D2000F583EBF0AF050D74002FF582E43400F588
:100D300083ECF07A007B00AF3A120F72AF3A020DEB
:010D4000BEF4
:0A0DF4008E2D8F2E8D2F8A308B314B
:100DFE00E4F532E532C3952F5020052EE52EAE2DAB
:100E0E007002052D14FFE5312532F582E43530F5FB
:0A0E1E0083E0FD120CFA053280D9C2
:010E280022A7
:0A0CB2008E2D8F2E8D2F8A308B318E
:100CBC00E4FDF532E53E6012E52DFF7E000DEE24DD
:100CCC0000F582E43400F583EFF0AE050D74002ED0
:100CDC00F582E43400F583E52EF07A007B00AF3A20
:0E0CEC00120F72AB31AA30AD2FAF3A020F5685
:100EBE0090E682E030E004E020E60B90E682E0303F
:100ECE00E119E030E71590E680E04401F07F147EF2
:0C0EDE0000120D4190E680E054FEF0226E
:10000E0090E682E044C0F090E681F0438701000064
:04001E0000000022BC
:100E8F0030040990E680E0440AF0800790E680E0A5
:100E9F004408F07FDC7E05120D4190E65D74FFF093
:0F0EAF0090E65FF05391EF90E680E054F7F02269
:08104700E4F51FD2E9D2AF224B
:100DBE0090E678E020E6F9C2E990E678E04480F02B
:100DCE00EF25E090E679F090E678E030E0F990E6F5
:100DDE0078E04440F090E678E020E6F990E678E09E
:060DEE0030E1D6D2E9223B
:100E5D00A90790E678E020E6F9E51F702390E67883
:100E6D00E04480F0E925E090E679F08D1AAF03A912
:100E7D0007751B018A1C891DE4F51E751F01D32200
:020E8D00C3227E
:100E2900A90790E678E020E6F9E51F702590E678B5
:100E3900E04480F0E925E0440190E679F08D1AAFAD
:100E490003A907751B018A1C891DE4F51E751F037B
:040E5900D322C322BB
:03004B00020607A3
:10060700C0E0C083C082C085C084C086758600C034
:10061700D075D000C000C001C002C003C006C0072B
:1006270090E678E030E206751F060206F190E6785C
:10063700E020E10CE51F64026006751F070206F162
:10064700E51F24FE605F14603624FE70030206E295
:1006570024FC70030206EE240860030206F1AB1BBC
:10066700AA1CA91DAF1E051E8F8275830012070FD6
:1006770090E679F0E51E651A7070751F05806B901E
:10068700E679E0AB1BAA1CA91DAE1E8E82758300FE
:1006970012073C751F02E51A6401704E90E678E078
:1006A7004420F08045E51A24FEB51E0790E678E061
:1006B7004420F0E51A14B51E0A90E678E04440F0AD
:1006C700751F0090E679E0AB1BAA1CA91DAE1E8E14
:1006D7008275830012073C051E800F90E678E04480
:1006E70040F0751F008003751F005391DFD007D0BE
:1006F70006D003D002D001D000D0D0D086D084D08D
:0807070085D082D083D0E032DE
:020EEA00A90756
:100EEC00AE18AF198F828E83A3E064037017AD0127
:100EFC0019ED7001228F828E83E07C002FFDEC3E79
:090F0C00FEAF0580DF7E007F00CE
:010F150022B9
:100F5600120E29E51F24FA600E146006240770F3AA
:0C0F6600D322E4F51FD322E4F51FD322B0
:100F7200120E5DE51F24FA600E146006240770F35A
:0C0F8200D322E4F51FD322E4F51FD32294
:100D41008E258F2690E600E054187012E5262401C6
:100D5100FFE43525C313F525EF13F526801590E63D
:100D610000E05418FFBF100BE52625E0F526E52528
:100D710033F525E5261526AE25700215254E6005AD
:060D810012002280EE22A8
:100022007400F58690FDA57C05A3E582458370F9F1
:0100320022AB
:03000000020AF7FA
:0C0AF700787FE4F6D8FD75813E020B3ECE
:10070F00BB010CE58229F582E5833AF583E022509F
:10071F0006E92582F8E622BBFE06E92582F8E222E9
:0D072F00E58229F582E5833AF583E4932203
:10073C00F8BB010DE58229F582E5833AF583E8F0F3
:10074C00225006E92582C8F622BBFE05E92582C89F
:02075C00F22287
:10075E00BC000BBE0029EF8DF084FFADF022E4CC7F
:10076E00F875F008EF2FFFEE33FEEC33FCEE9DEC48
:10077E00984005FCEE9DFE0FD5F0E9E4CEFD22ED8E
:10078E00F8F5F0EE8420D21CFEADF075F008EF2FD8
:10079E00FFED33FD4007985006D5F0F222C398FDC9
:0507AE000FD5F0EA2266
:1007B300D083D082F8E4937012740193700DA3A3D5
:1007C30093F8740193F5828883E4737402936860E9
:0607D300EFA3A3A380DFE9
:100FE700E4FFFE1207D9600C0FEF70010E09E970DC
:050FF700F20A80EF2268
:100B0300020A66E493A3F8E493A34003F68001F298
:100B130008DFF48029E493A3F85407240CC8C333F3
:100B2300C4540F4420C8834004F456800146F6DFC2
:100B3300E4800B0102040810204080900046E47E0C
:100B4300019360BCA3FF543F30E509541FFEE493B7
:100B5300A360010ECF54C025E060A840B8E493A37E
:100B6300FAE493A3F8E493A3C8C582C8CAC583CAA9
:100B7300F0A3C8C582C8CAC583CADFE9DEE780BE61
:01004A0000B5
:1007D900BB010689828A83E0225002E722BBFE021E
:0907E900E32289828A83E4932251
:00000001FF
